:020000040000FA
:0200000088284E
:08000800A02E071487148710D5
:10001000071008008710071487140800E80008304C
:10002000E9008710E81B871407140710E80DE90B97
:1000300011288316871483120714000007108316F3
:100040008710831208000830E90083168714831292
:100050000714031087180314E80D0710E90B28286C
:10006000831687108312680808008710071407108A
:100070008714080087140714071008000520D030E3
:100080000E20523004020E2000080E20840AE50BD8
:1000900044280A2008000520D0300E2052300402E7
:1000A0000E200520D1300E20562835202320800038
:1000B000840AE50B55283A200A2008000030E600A3
:1000C0007630E7001230E5000520D0300E20722097
:1000D0008A110A120E20E70A0319E60AE50B6728BF
:1000E0000A20080066088A0067088200003400348D
:1000F0000034003406340134013421340034003437
:10010000003400340034003400340034003400344F
:10011000031383122030A20083018B018501870124
:1001200007309900831691013F3085000030870029
:100130003730950071308F00433081000C108312EE
:1001400001309000C0308B000B3087003C214526E9
:10015000051CAE28D126F2263C2779210930C200A1
:10016000DB30C30058210A30C7000830CA004A08F3
:10017000C2004703C30006304A020319C30103301B
:100180004A020319C3015821CA0BB7289626C70B88
:10019000B52879210930C2005830C3005821732195
:1001A0000730C2000130C30058210630C200403081
:1001B000C30058210530C2000030C300582104306C
:1001C000C2000130C30058219A2679216130840091
:1001D0000130E5004B20E11F22290930C2001B300D
:1001E000C30058210830C2004F30C30058210730E7
:1001F000C2008530C30058210630C2000030C30061
:1002000058210530C2000330C30058210430C20019
:100210000230C30058210330C2000030C30058210F
:100220000230C2000330C30058210130C200013047
:10023000C30058215C263B3005053B3A03191B29B6
:100240005E20E628AE01CF01CE01AD018030B100C5
:10025000523084000730E5004B203321A621AE1731
:10026000A1010B168429FF30A300A400A500A6005D
:10027000A700A800A90008000F30C2000030C3008A
:1002800058210930C2000030C30058210A30C20092
:100290000430C300CD0058210B30C2000730C3002A
:1002A00058210C30C2000130C300582173210800CE
:1002B00087114208662143086621871508008711C7
:1002C000420866210301662187150800C400083032
:1002D000C5000711C41B0715071600000712C40D3F
:1002E000C50B692908000830C2005F21C20B7529BF
:1002F00008000C30C200C301582198260C30C200FF
:100300000130C30058210800AE1B8829211C9D29FB
:10031000523084000730E5004B20A621AE132E0892
:100320000319EB2401302E0203196E2502302E0230
:100330000319BB25211000261226051C1C22851C32
:100340000F23851E1923851D9F238429D001D101E8
:100350002808B8005208A8005014F0393806F039BF
:100360000319062AD0142708B8000F3953060F398D
:100370000319062A5308A7005015F0393806F0393A
:100380000319062AD0152608B8000F3954060F396C
:100390000319062A5408A6005016F0393806F03919
:1003A0000319062AD016550829060319062A5508E6
:1003B000A90051142508B8005608A500D114F03939
:1003C0003806F0390319062A51152408B8000F39E8
:1003D00057060F390319062A57081F39A400D115EB
:1003E000F0393806F0390319062A51162308B800E7
:1003F0000F3958060F390319062A5808A300D116D9
:10040000F0393806F0390319062A5117AE1F0C2AA5
:100410007E30D1003F30D00008002808D2002708E5
:10042000D3002608D4002908D5002508D6002408C2
:10043000D7002308D80008007F260518A92A3C30D9
:10044000BB0081267F302E05031D302A211C302A57
:10045000523084000730E5004B20A621EB24211008
:100460000518352ABB0B212A3C2AAE0A03302E027E
:100470000319AE01AE17A92A0B120930C200DB30F6
:10048000C30058210830C2000A30C3005821073089
:10049000C2000A30C30058210630C2000030C30039
:1004A00058210530C2000A30C30058210430C20070
:1004B0000A30C30058210330C2000030C300582165
:1004C0000230C2000A30C30058210130C2000A3095
:1004D000C3005821051C6A2AAF01B001A1010630F2
:1004E00081006430A0008B16301003302F020318F7
:1004F0007F2A7E30D100AF0A6E25AF03842A3F30B9
:10050000D000AF0AEB24AF03051CAC22851CB5223A
:10051000051EDB22851E012306302F020319982AAF
:1005200003303005031D742ACF1C842ACF10742A8F
:100530008B12CF01051C9A2AB01CA42A0D2252301E
:1005400084000730E5003E20AF01B001AE01AE17D8
:100550000B16051CA92A08007F260518B12A30149D
:10056000AF0A051CB12A7F2608007F268518D92AE4
:10057000B0142F08031DBE2A0124C92A01302F02FE
:10058000031DC42AF723C92A02302F02031DCC2AD7
:10059000AC237C24A900D92A03302F02031DD22AC0
:1005A0004324D92A04302F02031DD82A3B24D92AF8
:1005B0003324852608007F26051AFF2AB0142F0849
:1005C000031DE42A2424EF2A01302F02031DEA2A06
:1005D0001824EF2A02302F02031DF22A0A247C2459
:1005E000A900FF2A03302F02031DF82A5F24FF2AE7
:1005F00004302F02031DFE2A5524FF2A4B24852692
:1006000008007F26851A0B2B3014AF032F0A031D19
:100610000B2B0530AF00851E0B2B7F2608007F2695
:100620008518152B0230AD06AE17851C152B7F26BD
:1006300008007F26851A422B05302702031C372B22
:1006400055302702031C462B0B1243242608031D9A
:10065000382BAC2301302502031D342BF723013046
:100660002402031D342B01247C24A900382B0B12F7
:10067000A701A8010D22523084000730E5003E207A
:100680000B16AE17851E422B7F260800211C502B0F
:10069000523084000730E5004B20A62121105E2B4C
:1006A0004F1D562BCF1C692BCF105A2B2F08031927
:1006B000692BAF013F30D0007E30D1002E080319E6
:1006C000EB2401302E0203196E2502302E0203198D
:1006D000BB25851C8623051E9323CD1F7F2BCD13A1
:1006E0000A30C2004D08C30058210530CE00073043
:1006F000CF00063081006430A0008B16502B851E81
:10070000462BAF01CF01AE173321422B7F26851830
:100710008F2BCD0A0A304D020318CD03CD17851C4F
:100720008F2B7F2608007F26051A9B2BCD034D0AB1
:100730000319CD01CD17051E9B2B7F2608007F26B0
:100740008519A82B8030B106B11B3826B11F55265C
:10075000851DA82B7F260800B7232502031DB32B78
:100760000130A500B62B2530840069240800023032
:100770002402031DC62B2308B4002208B300DA2389
:10078000321CC42B2930D92B2830D92B0430240219
:100790000319D82B063024020319D82B0930240260
:1007A0000319D82B113024020319D82B3130D92B3F
:1007B00030300800B2013408EA230339031DE92B65
:1007C0003408031DE82B3308EA230339031DE92B02
:1007D00032140800B900390E0F39B8000310B80DF3
:1007E000B80DB807B80D39080F393807080024309C
:1007F0008400692413302402031D002C0130A4005E
:100800000800233084006924A0302302031D092C32
:10081000A3010800A503031D102CB723A500172C66
:1008200025080F390F3C031D172C0630A5020800C0
:10083000A403031D1D2C1230222C0F302402031D93
:10084000232C0930A4000800A303230A031D2B2C2A
:100850006630A302322C23080F390F3C031D322CC3
:100860000630A30208002830840069246030280282
:100870000318A8010800273084006924603027028B
:100880000318A701080026308400692424302602BA
:100890000318A6010800283084007224F9302802C9
:1008A000031D542C5930A8000800273084007224FE
:1008B000F9302702031D5E2C5930A70008002630AE
:1008C00084007224F9302602031D682C2330A60010
:1008D0000800800A00080F390A3C031D0800063092
:1008E0008007080000080F390319782C80030800DE
:1008F00080030630800208000130B400B3010130EB
:10090000B6002208EA23B70004303702031C902CFB
:10091000031D8D2C23080319902C0430B702842C5E
:1009200023083402031D982C370833020319AD2C19
:100930000130B607DA233218B60A07303602031838
:10094000B600343084006924A0303402031D902C9A
:10095000B401333084006924902C0130B5002408A0
:1009600035020319C72C3508EA23B900D424B60789
:1009700002303502031DBF2CDA233218B60A0730C5
:1009800036020318B600353084006924AF2C2508E0
:10099000EA23B607B60307303602031CD12CB60093
:1009A000CB2CB60A360808003903CC000430CB0043
:1009B000E030CC070318CB0A4B088A004C088200B1
:1009C0000334003403340234033402340334033474
:1009D00002340334023405304F19AF000930C2002D
:1009E000DB30AD185B30C30058210130C20028084D
:1009F0000F39C30006304825D01C3D2D0230C200FF
:100A0000280E0F39C30006304825501D3D2D0430F7
:100A1000C20027080F39C3004D084F19C300053025
:100A20004825D01D3D2D0530C200270E0F39C300CB
:100A30004D084F19C30005304825501E3D2D26088E
:100A4000AA00AD1854250730C2002A080F39C30088
:100A5000043048250830C200AD18322D2A0E0F3957
:100A6000C3003B2D2A08F039031D3030C30002308B
:100A70002D180430C30404304825D01D472D033001
:100A8000C2006030C30058210630C200582108005F
:100A9000AF080319522D4F1C522D2F02031D522D4A
:100AA0008030C304582108002D102A08031D5B2D37
:100AB0001230AA006D2D12302A02031C6D2D2D1448
:100AC00003196D2DAA000E302A02031C6D2D103063
:100AD0002A0203186D2D0630AA02080002304F19B1
:100AE000AF00D11CBA2D0930C200DB30C300582141
:100AF0000130C20025080F39C30003304825511DBD
:100B0000B22D0230C200250E0F39C3000330482534
:100B1000D11DB22D0430C20024080F39C3004D0886
:100B20004F19C30002304825511EB22D0530C200B6
:100B3000240E0F39C3004D084F19C3000230482559
:100B4000D11EB22D0730C20023080F39C300013077
:100B50004825511FB22D0830C200230E0F39C300A3
:100B6000013048250330C2004030C3005821063010
:100B7000C2005821080010302802031CD62D203056
:100B80002802031CCF2D30302802031CD62D403004
:100B90002802031CCF2D50302802031CD62D280814
:100BA0000F397E300319D1006E25DC2D28080F394E
:0A0BB0003F300319D000EB240800C9
:100C0000B11F112E59302702031D0C2E5730280218
:100C1000031C0C2E3115112E28082704031D112E3C
:100C2000B11508007F3031050319262E311C1A2E0C
:100C30004326242EB11C1F2E55265526242E311D49
:100C4000232E2726242E2E268030B1050800F730CB
:100C5000BD001F30BE0064306026080031263126FA
:100C60003126FB30BD009030BE00FA30602608000F
:100C70003C267F263C267F26F630BD000930BE008C
:100C800064306026080045267F263C267F26F83003
:100C9000BD008930BE00643060260800F130BD0020
:100CA0001230BE00643060260800F130BD00123002
:100CB000BE00FA30602608004E268326552608001E
:100CC00083160C148312882683160C1083120800D6
:100CD0000430BF000000BF0B6A2E000008000F3078
:100CE000BF00722EBF0B712E752E08002730BF007B
:100CF000792EBF0B782E7C2E08000A30882E1E30ED
:100D0000882E3230882E6430882EC830882E0130EC
:100D1000C000DD30BF008C2E8D2E8E2EBF0B8B2E93
:100D20000000922E932EC00B892E080005309B2EBA
:100D30000A309B2E3230C1008326C10B9C2E080046
:100D4000FD00030EFE000408FF0083128B18AD2E79
:100D50000B19B02E0C18C32ECA2E8B102114CA2EBC
:100D60000B1106308100A00BCA2E0130CF06CF1424
:100D7000CE080319C02ECE03031DC02E8B12CF0147
:100D80006430A000CA2E0C103D088F003E088E0073
:100D9000203087067F0884007E0E8300FD0E7D0EC6
:100DA00009000230C6000830C200063042020319B2
:100DB000C203033042020319C2034030C3000730AC
:100DC000C900582185265F210310C30CC90BE12EF1
:100DD0008030C300582185265F21C20BD52EC60B5B
:100DE000D32E08000330C6000830C2000330C7000D
:100DF0004030C3000230C800582183265F21C2035F
:100E0000C80BFC2EC20A0230C8000310C30C5821C4
:100E100083265F21C80B052F0310C30C0230C800C6
:100E2000582183265F21C20AC80B102FC20302304B
:100E3000C8000310C30C582183265F21C80B192F4B
:100E40000310C30C0230C800582185265F21C2035D
:100E5000C80B242FC20A0314C30C0230C800582147
:100E600085265F21C20AC80B2F2F0430C202C70B90
:100E7000F82EC60BF42E08000330C6000830C2005E
:100E80004030C3000630C800582183265F21C203CA
:100E9000053048020319C203033048020319C20394
:100EA000C80B442FC20A0230C8000310C30C5821DB
:100EB00083265F21C80B552F0310C30C0630C800D2
:100EC000582183265F21C20A033048020319C20A4F
:100ED000053048020319C20AC80B602FC203023052
:100EE000C8000310C30C582183265F21C80B712F43
:100EF0000310C30C0630C800582183265F21C203AB
:100F0000053048020319C203033048020319C20323
:100F1000C80B7C2FC20A0314C30C0630C80058212A
:100F200085265F21C20A033048020319C20A053030
:100F300048020319C20AC80B8F2FC60B3E2F0800A8
:02400E00C43CB0
:1042000043006F0070007900720069006700680069
:1042100074002000280043002900200032003000F4
:104220003200310020006200790020004D002E0095
:10423000590061006D0061006D006F0074006F0037
:02424000FF007D
:00000001FF
